:1000000001C0D7C030E838B937E037BB33E038BB80
:1000100031E031BB35E032BBF0E070E0872E50E4D8
:100020007EBB6FD13DB3CBD173955A95C9F788206C
:1000300019F0F2603FE031BD32E035BF30E43BBF44
:100040007894A4C02227A895F1FDC29A2223D9F35F
:100050002227CD2F69D1D13409F40DC0D33409F44E
:1000600021C0D43409F433C0D33509F447C0DA359C
:1000700009F468C080C069D1D770DD2309F47BC062
:10008000DA957D2F770F770F770F86E0780FE1E015
:1000900063D18DBB7EBB39D173955ED18DBB7EBBE9
:1000A00034D159C052D1D770DD2309F464C0DA9538
:1000B0007D2F770F770F770FE1E050E085E58DBB5F
:1000C0007EBB23D1739553955830C1F744C0CDE022
:1000D0002BD1CAE029D150E0952F977021F4CDE0C3
:1000E00023D1CAE021D15EBB0CD18DB312D114D182
:1000F000C0E21AD15395583379F748C026D1D7704A
:10010000DD23C9F1DA95AD2EF160A895F0FDFDCFA4
:10011000C1E30AD156E0E1E07A2D770F770F770F30
:10012000C198C19A30813DBB7EBBEFD0E3957395FA
:100130005A95B1F735E03DBB7EBBE7D073957EBBEA
:10014000E4D009C070E05FE37DBB7EBBDED0739579
:100150005A95D9F700C070E0872E5FE37EBBD1D0FF
:100160003DB32DD173955A95C9F78DBA7EBBCDD0CD
:10017000FD7FC29803C0CAE2D7D008C0CDE0D4D07A
:10018000CAE0D2D0CFE4D0D0CBE4CED0CDE0CCD03A
:10019000CAE0CAD0C5E4C8D0CDE2C6D0CBE4C4D052
:1001A000C5E6C2D0C9E7C0D0CEE3BED03FE031BD86
:1001B00049CF9FB6819BE9C08299A1C004E011EAB2
:1001C0001A95F1F70A95D9F733E347E08A9A92989E
:1001D0001AE01A95F1F7379508F4929A0AE019E0B7
:1001E0001A95F1F70A95D9F7929A1AE01A95F1F74C
:1001F0004A956AF71FEF1A95F1F7E0E058E048E0FA
:10020000129A929813E01A95F1F71298929A1AE0BE
:100210001A95F1F788948299089437951EE01A95FB
:10022000F1F71EE41A95F1F74A9551F73083E395FB
:100230005A9529F7E0E058E088243081C0D0E39552
:100240005A95D9F7882019F0C3E26ED058C0CDE096
:100250006BD0CAE069D0E0E08E2F8F7021F4CDE042
:1002600063D0CAE061D0808154D056D0C0E25CD067
:10027000E395E73089F7CDE057D0CAE055D0A8958F
:10028000F0FD3CC0F1FD3AC070E0E1E080E056E0F6
:10029000870F8EBB36D03DB39081931759F5E39508
:1002A00083955A95B1F78EBB2CD09DB383958EBBA9
:1002B00028D0ADB3992309F0C098AA2309F0C198BA
:1002C000B0E1A89500EA1FEF1A950000E9F70A953A
:1002D000D1F7BA95B1F7992319F09A9509F4C09A14
:1002E000AA2319F0AA9509F4C19A992349F7AA23D8
:1002F00039F704C098E0790F783339F6FE7F9FBE56
:100300001895E09AE099FECF0895E19AE199FECF21
:100310000895C82FC29502C0C82F00C0CF70CA5F11
:10032000C4FDC95FC65D00C0BBE0BB3021F0B33087
:1003300020F0C79510F0909A01C0909814E61A9595
:100340000000E9F7BA9589F70895A8952223E9F303
:100350002227CD2FE9DF0895A8952223E9F322274C
:10036000CD2FE2DFD053DA300AF0D750DF70D295CC
:100370008D2FA8952223E9F32227CD2FD5DFD05347
:10038000DA300AF0D7508D2B0895B9E012E31A95B0
:100390000000E9F7889481990894909A9098D795ED
:1003A00012E31A950000E9F7BA9581F721E09FBEA4
:1003B0000EE11EE11A95F1F70A95D9F71895A32FCA
:1003C00048E03A2F38253795382D10F498E1392731
:1003D0003795832E3A2F3695A32F4A9591F7089596
:00000001FF
